:020000040800F2
:1000000008040020D500000843020008410200084F
:1000100000000000000000000000000000000000E0
:100020000000000000000000000000006502000861
:100030000000000000000000450200086702000800
:100040000501000805010008050100080501000878
:100050000501000805010008050100080501000868
:100060000501000805010008050100080501000858
:100070000501000805010008050100080501000848
:100080000501000805010008050100080501000838
:100090000501000805010008050100080501000828
:1000A0000501000805010008050100080501000818
:1000B0000501000805010008050100080501000808
:1000C0000348854600F032F8004800477D030008E9
:1000D000080400200C4880F308880C480168090EC9
:1000E0000B4A914205D10B480B4901600B480C4962
:1000F00001600C4880470C480047FEE7FEE7FEE73A
:10010000FEE7FEE7FEE70000080400200400000010
:100110001F00000018100240010000000000014014
:100120000000000069020008C1000008064C01251B
:10013000064E05E0E36807CC2B430C3C984710348F
:10014000B442F7D3FFF7C0FFF00300080004000833
:10015000F0B584B00A68002302240092039116E0EF
:100160000168029D29400160A240016811430160BD
:10017000C1682940C160039DE979A140C2680A4372
:10018000C2602946009A241D9B1C102B56D00126C4
:1001900035469D402A4231D0A71E03220297BA401D
:1001A000D24301920A79511E012913D88168019F17
:1001B0003940816003994979029FB94087680F43AC
:1001C00087608188A94381800399897999408588CE
:1001D0000D4385800168019D29400160029FBA405E
:1001E000016811430160C1682940C160039DE9793C
:1001F000B940C2680A43C2602946009A5F1CBE40EB
:100200003242C0D00322A240D24302920A79551E44
:10021000012DA5D8856802990D40856003994D7917
:10022000A5408168294381608188B1438180039919
:100230008979B94085880D43858091E704B0F0BD88
:10024000FEE7704770470000054A002903D0116897
:100250000143116070471168814311607047C046C7
:10026000141002407047704770B582B03F48011FBC
:100270000B68012213430B6003683D4C1C40046073
:100280000B683C4C1C400C6093040C689C430C6055
:100290003F231B0404689C430460836A0F24A34328
:1002A0008362FF235433C46A9C43C462036B934349
:1002B0000363002343600193009314040D682543F6
:1002C0000D6054040D6825400095019D6D1C01953D
:1002D000009D002D04D105252D03019EAE42F1D1D4
:1002E0000D68254201D1009300E00092009B012B94
:1002F00039D1214B11241C6003680360036803603B
:100300007F23DB0305689D430560230404681C43C9
:10031000046013060C681C430C6052060B68134201
:1003200008D10B68134205D10B68134202D10B6848
:100330001342F3D001680322914301600168022255
:100340000A43026002680C210A40082A0BD00268A6
:100350000A40082A07D002680A40082A03D0026827
:100360000A40082AEED102B070BDC0460410024017
:100370000CB8FF08FFFFF6FE002002400121C80470
:10038000FFF762FF032084020E490F480C604860AB
:100390000E4D28461838FFF7DBFE2C602C822C60AF
:1003A0002C822C602C822C602C822C602C822C6065
:1003B0002C822C602C822C602C822C602C822C6055
:1003C0002C82EAE700000020010300001808004822
:1003D00002E008C8121F08C1002AFAD1704770470E
:1003E000002001E001C1121F002AFBD1704700006C
:1003F000000400080000002008040000E0030008DA
:04000005080000C12E
:00000001FF
